:1000000028288F018E00FF308E07031C8F07031CEA
:10001000232803308D00DF300F2003288D01E83EB8
:100020008C008D09FC30031C18288C070318152838
:100030008C0764008D0F15280C181E288C1C222894
:1000400000002228080083130313831264000800B1
:1000500006108316061083128610831686108312EC
:1000600006118316061183128611831686118312D8
:1000700006128316061283128612831686128312C4
:1000800006138316061383120F308F00A030022050
:100090006120C83001206E206E20AF20AF20AF203D
:1000A0006E2061207B20A22061208820AF2061206B
:1000B0006E207B20AF2061207B2095206120630093
:1000C0005F28061783160613C83083120120061313
:1000D00083160613C8308312012008000614831605
:1000E0000610C83083120120061083160610C8308F
:1000F000831201200800861483168610C8308312EC
:100100000120861083168610C83083120120080053
:10011000061583160611C8308312012006118316B6
:100120000611C83083120120080086158316861137
:10013000C83083120120861183168611C8308312BD
:1001400001200800061683160612C830831201200B
:10015000061283160612C830831201200800861684
:1001600083168612C83083120120861283168612E7
:08017000C830831201200800D1
:02400E00F53F7C
:00000001FF
